:020000040000FA
:1002000099EF01F09EA8FED70A50AD6E1200ABA286
:1002100002D0AB98AB889EAAFED7AE500A6E1200F1
:1002200089688A6A8B68F00E926E3F0E936E9F0EFD
:10023000946EC60EC16EC00EC26E400EAF6EFB0E47
:10024000AC14AC6E200EAC10AC6E100EAB10AB6EDE
:10025000800EAB10AB6E03680F0E046E016A815006
:10026000056E05B222D0066A076A086A096A0404A4
:10027000046E0450896E0950000808E10850070810
:1002800005E10750A10802E10650200802E209AE8C
:1002900008D0062AD8B4072AD8B4082AD8B4092A1C
:1002A000EAD7110E0124016E23D005B821D0066AC9
:1002B000076A086A096A0428046E0450896E0950A6
:1002C000000808E10850070805E10750A10802E10D
:1002D0000650200802E209AE08D0062AD8B4072A40
:1002E000D8B4082AD8B4092AEAD7110E015C016EE5
:1002F0000368026807EC01F00A50026E02B003D0F6
:10030000FD0E0314036E02B203D0FB0E0314036E42
:1003100002B403D0FE0E0314036E02B603D0F70E30
:100320000314036E0350896E01500A6E02EC01F053
:0603300096D710EF01F06A
:020000040030CA
:0E000000FFFEF6FEFFFEFBFFF03FFF9FFFBF7F
:00000001FF
